:020000040800F2
:1000000000040020E1010008E3010008E20100080B
:10001000E2010008E2010008E2010008E201000834
:10002000E2010008E2010008E2010008E52C0008F6
:10003000E2010008E2010008E2010008E201000814
:10004000E2010008E2010008E2010008E201000804
:10005000E2010008E20100084D2F0008792F000896
:10006000A52F0008D12F0008FD2F0008E20100088D
:10007000E2010008E2010008E2010008E2010008D4
:10008000E2010008E2010008E2010008E2010008C4
:10009000E2010008E2010008E2010008293000083E
:1000A000E2010008E2010008E2010008E2010008A4
:1000B000612D0008E2010008E2010008E2010008E9
:1000C000E2010008E2010008E2010008E201000884
:1000D000E2010008E2010008E2010008E201000874
:1000E00091300008E2010008E2010008E201000886
:1000F000E2010008E2010008E2010008E201000854
:10010000E2010008E2010008E2010008E201000843
:10011000E2010008E2010008E2010008E201000833
:10012000E2010008E2010008E2010008E201000823
:10013000E2010008E2010008E2010008E201000813
:10014000E2010008E2010008E2010008F1230008D2
:10015000E2010008E2010008E2010008E2010008F3
:10016000E2010008E2010008E2010008E2010008E3
:10017000E2010008E2010008E2010008E2010008D3
:10018000E2010008E2010008E2010008E2010008C3
:10019000E2010008E2010008E2010008E2010008B3
:1001A000E2010008E2010008E2010008E2010008A3
:1001B000E2010008E2010008E2010008E201000893
:1001C000E2010008E2010008E2010008E201000883
:1001D000E2010008E2010008E2010008E201000873
:1001E00002E000F000F8FEE772B6384880F30888B5
:1001F000374880F3098837484EF60851CEF200019F
:10020000086040F20000CCF200004EF63471CEF2ED
:1002100000010860BFF34F8FBFF36F8F40F2000003
:10022000C0F2F0004EF68851CEF200010860BFF334
:100230004F8FBFF36F8F4FF00000E1EE100A4EF6C4
:100240003C71CEF200010860062080F31488BFF3F1
:100250006F8F01F095FD02F0DDFC1F481F491B4A1E
:1002600091423CBF41F8040BFAE71D49184A9142FC
:100270003CBF41F8040BFAE71A491B4A1B4B9A4250
:100280003EBF51F8040B42F8040BF8E70020184970
:10029000184A91423CBF41F8040BFAE701F074FDA3
:1002A00002F014FD144C154DAC4203DA54F8041B53
:1002B0008847F9E700F040F8114C124DAC4203DAE0
:1002C00054F8041B8847F9E701F05CBD00040020E6
:1002D000000800200000000855555555000000207A
:1002E00000040020683500080008002028080020CD
:1002F00028080020F0170020E0010008E0010008B5
:10030000E0010008E00100082DE9F04F2DED108A12
:10031000C1F80CD0C3689D46BDEC108ABDE8F08FD3
:10032000002383F311882846A047002001F0E4F958
:1003300001F094F900DFFEE738B5184B6FF07A0250
:1003400000241A700F225C709C70DC701C715C7150
:100350009C71DC711C725C729A72DC7201F0EEFCB2
:100360000F4B984208D00133984241F2883412BFB3
:1003700000250024012500E02546002001F0E4FCD2
:100380000DB100F053F800F063FC00F03BFB204699
:1003900000F0A0F800F04AF8F9E700BF28080020B4
:1003A000010007B008B500F0CBFAA0F120035842D5
:1003B000584108BD07B5054B01A81B88ADF80430AE
:1003C000022100F00FFB03B05DF804FB3832000897
:1003D00008B51248C3680BB101F014FA104A0F486F
:1003E00000234FF47A7101F0D1F90E4B1A6812B163
:1003F0001A68013A1A605A680A4912B14A68013A01
:100400004A60094A12783AB95B682BB9022000F0B9
:10041000D9FB044B32225A6008BD00BF34080020CB
:10042000D10300084C0D0020480D002038B5224CA7
:10043000236801333ED0214D214B2A689A4239D995
:10044000204B9B6803F1006303F580339A4231D25D
:10045000002000F0F1FA1C4B0220187000F0A8FBFD
:100460001A4B1A6C00221A64196E1A66196E596CAE
:100470005A64596E5A665A6E5A6942F080025A613D
:100480005A6922F080025A615A691A6942F0005290
:100490001A611A6922F000521A611B6972B60C4B7C
:1004A0001C6023682A68202181F311889D4683F30C
:1004B0000888104738BD00BF00000108040001088B
:1004C000FFFF000828080020480D002000380240E7
:1004D00008ED00E02DE9F04FBE4B8046BE489C6819
:1004E0000022C26091B0202282F31188C268019379
:1004F0000AB101F087F9B848B84A4FF47A7100237D
:1005000001F044F9002383F31188DFF8ECA2B8F17D
:10051000000F01D0CAF80080B14ECAF8043000259F
:100520003370A9464FF0FF37012000F041FBB8F1CE
:10053000000F04D0DAF80030002B00F0F781002023
:1005400000F0FEF90590059B002BF0DB012000F088
:1005500025FB059B213B122BE6D801A252F823F084
:10056000AD050008BF0500082B0600082905000896
:1005700029050008290500089F060008290500082C
:100580004F070008FD0700082B0800085508000861
:10059000290500086B0800082905000895080008CF
:1005A000F908000829050008C50800080220FFF71F
:1005B000F9FE002800F0A7814FF001099CE14FF4FB
:1005C0007A7000F0BDF9B0F1000BC0F29C810220FE
:1005D000FFF7E8FE002800F096810BF1FF300428B9
:1005E00000F29181DFE800F003080A0C110010A866
:1005F000052340F8143D04E0764802E0794800E025
:100600007948042100F0EEF90DE01C25284600F0A1
:1006100015FA10AB042143F8140D0435184600F008
:10062000E1F92C2DF2D1012566E1B9F1000F00F0BE
:100630006A81002D00F067810220FFF7B3FE10B938
:100640000125A9465FE1012000F0F6F90220307093
:1006500000F0AEFA0024E3B21846029300F004FA68
:1006600001348346029B18B1184600F00DFAF2E7F8
:1006700001230220337000F091FA019B9B689B4597
:1006800008D2584600F0DAF9013040F045810BF10C
:10069000040BF2E700243470CAF804402CE1B9F1ED
:1006A000000F00F03081002D00F02D81022030700D
:1006B00000F07EFA322000F043F9B0F1000BBFDB0E
:1006C0001BF00303BCD1019989680BEB04028A4239
:1006D000B6D8BBF5807FB3D85B450EDA4FF47A709D
:1006E000029300F02DF90590059A002AA8DB029BE1
:1006F0003E4A059999540133EEE7C820FFF752FEB0
:1007000000289DD024B9394B4FF0FF321F681A6082
:100710002BF0030B0BEB0403A3469B4515D0334A88
:100720000393121B584652F80B10029200F08CF9FA
:10073000584600F083F9029A52F80B20904240F09C
:10074000EB800BF1040B039BE7E75C46D4E002204F
:10075000FFF728FE002800F0D6804FF00008C346BF
:10076000019B9B68984530D2B8F1000F03D17A1CE9
:1007700001D00B9703E0404600F060F90B901C4954
:100780004B6893B91A46082012F0010F4FEA520E37
:1007900016BF184A72468EEA02020138F4D141F8B7
:1007A00023200133B3F5807FECD100220BABD35C67
:1007B00083EA0B03DBB2013251F82330042A83EAC7
:1007C0001B2BF3D108F10408CAE710A840F828BD94
:1007D00029E000BF2808002034080020D1030008C9
:1007E000480D00202C08002030080020480C002074
:1007F000480800202083B8ED4C0D002010A80023ED
:1008000040F8143D642100F0C7F800287BD1022095
:10081000FFF7C8FD002876D00B9800F047F910AB21
:1008200043F8240D1846042131E010A8002340F8B5
:10083000143D642100F0B0F8002864D10220FFF7D5
:10084000B1FD00285FD00B9800F040F910AB43F8E1
:10085000200DE7E70220FFF7A5FD002853D000F0A8
:100860003BF910AB43F81C0DDCE70220FFF79AFDC3
:10087000002848D00BA9142000F034F9804610A8B5
:10088000042140F8188D00F0ADF80BA8414600F0A7
:10089000A9F831E04FF47A70FFF784FD98B37B1C20
:1008A00005D1FFF787FD234800F02CFF3EE0002034
:1008B000394600F0C9F8002000F0C0F8B842F0D086
:1008C000A34629E010A8002340F8143D642100F05D
:1008D00063F88346B8B90220FFF764FD98B1FFF7CB
:1008E00069FD41F2883000F00DFF0B9800F0DAF955
:1008F000D84600F0A3F917E600F0A0F94FF0000881
:10090000FFF758FD10E60C4B0BA81B88ADF82C30F8
:10091000022100F067F807E6084B0BA81B88ADF82A
:100920002C30022100F05EF85C46FDE511B0BDE818
:10093000F08F00BFA08601003A3200083C32000868
:1009400073B5124B1A780132D2B20024012A06463E
:100950008DF8074010D80E4803681D6A4FF47A736B
:100960000DF1070101227343A847012804D1094B67
:100970009DF807001C7005E04FF4FA7000F0C2FE0D
:100980004FF6FF7000B202B070BD00BF000800203B
:10099000B00D0020540D002038B50F4A12780132F6
:1009A000D2B2012A03460D460ED80C4802681946F9
:1009B0004FF47A73146A6B430422A047042803D1CE
:1009C000074B0020187038BD4FF4FA7000F09AFE03
:1009D0004FF0FF3038BD00BF00080020B00D0020F0
:1009E000540D002010B5034604480A460168CC693E
:1009F0001946A446024BBDE810406047B00D0020E8
:100A0000A086010070B501F0C3F8094B00261870EC
:100A10001C46084D23782868984208D201F0B2F8A5
:100A20002B6806440133B6F5803F2B60F1D370BDCF
:100A30005C0D0020580D002001F06CB900F1006041
:100A400000F580300068704707B502AB00F1006028
:100A500043F8041D0422194600F5803001F0DCF84B
:100A600003B05DF804FB0000054B1A68054B1B78CA
:100A70001344984202D2104401F084B80020704719
:100A8000580D00205C0D002038B5074D044628683D
:100A9000204401F07FF828B928682044BDE8384098
:100AA00001F090B838BD00BF580D0020034610F08B
:100AB000030008D1B3F5007F06D803F10053A3F576
:100AC000084318687047002070470000014BC05869
:100AD000704700BF107AFF1F014B1868704700BFB6
:100AE000002004E070B52A4B1C68C4F30B03240CEF
:100AF00083B140F21342934209D040F2194293422B
:100B000007D040F2214293420BD1032302E001239C
:100B100000E002231F4A0C2505FB03235D681A7AB7
:100B200001E01D4D3F2242F201039C422CD0B4F55E
:100B3000805F08D041F201039C420BD041F20303D5
:100B40009C4209D000E0412241F207039C4208BFC9
:100B5000312202E05A2200E05922461E0E44013D95
:100B60000C46B4420ED215F8010F631C18B11C4696
:100B700003F8010CF5E72C20B342207006D2A31C29
:100B8000627003E0234601E03322DDE7581A70BDAE
:100B9000002004E04032000870320008022802BF42
:100BA000024B4FF080729A61704700BF0000024014
:100BB000022802BF024B4FF480729A61704700BF57
:100BC00000000240022801BF024A536983F4807387
:100BD000536170470000024010B50023934203D0D8
:100BE000CC5CC4540133F9E710BD000030B50138C6
:100BF00010F8013F0C4663B12578AB4201F10101C9
:100C000007D10AB1013AF3E75AB294F90030D01A89
:100C100030BD002AF8D1104630BD00000246034620
:100C2000981A13F9011B0029FAD1704702440346B0
:100C3000934202D003F8011BFAE77047024B1A787F
:100C4000024B1A70704700BF540D002000080020AE
:100C500038B5104D104C284600F0A4F8214628461F
:100C600000F0CCF823680D485A6DD2F8043843F0F0
:100C70000203C2F8043800F045FD2068084900F07E
:100C8000C5F923685A6DD2F8043823F00203C2F87C
:100C9000043838BDB00D0020D433000840420F00A6
:100CA0006833000870470000026843681143016020
:100CB00003B11847704700000020704713B5446B1C
:100CC000D4F894341A681178042916D1217C0229A9
:100CD00013D11979128901238B4013420DD104F1EC
:100CE0004C0001A901F0F8FD024630B1D4F894346B
:100CF00018681979019B00F0D5F902B010BD000009
:100D0000143001F067BD000014304FF0FF3301F0E4
:100D100061BD00004C3001F04DBE00004C304FF082
:100D2000FF3301F047BE0000143001F037BD000072
:100D300014304FF0FF3101F031BD00004C3001F0B4
:100D400019BE00004C304FF0FF3201F013BE00001E
:100D5000D0F8942438B5136819780429054601D0D1
:100D6000012038BD017C0229FAD112795C89012069
:100D700090400440F4D105F1140001F0C5FC024696
:100D80000028EDD0D5F89434186859794FF4807361
:100D900000F076F9204638BD406BFFF7D9BF000060
:100DA000704700007FB5124B0360002343608360EF
:100DB000C3600446012502260E4B057429460193A3
:100DC000029004F18402009614304FF4807301F015
:100DD00077FC094B01930096029404F14C002946DC
:100DE00004F523724FF4807301F052FD04B070BD1E
:100DF0009C320008990D0008BD0C00080B682022E9
:100E000082F311880A7903EB820290614A790932F0
:100E100043F822008A7912B103EB8203986102231E
:100E20000374C0F89414002383F311887047000002
:100E300038B50446012504300221FFF735FF04F1DF
:100E4000140025776FF0010100F084FC84F8545001
:100E500004F14C006FF00101BDE8384000F07ABCAD
:100E600010B5012104460430FFF71EFF002323774D
:100E700084F8543010BD000038B504460025143005
:100E800001F036FC04F14C00257701F019FD201D1E
:100E900084F854500121FFF707FF2046BDE8384091
:100EA000FFF756BF90F8443003F06003202B19D1B0
:100EB00090F84520212A0AD0222A4FF000030CD0B6
:100EC000202A0FD1084A82630722C26307E0064B3B
:100ED00083630723C363002301E08363C363036465
:100EE000012070470020704701080020D0F894349A
:100EF00037B51A681178042904461AD1017C0229F1
:100F000017D11979128901238B40134211D100F1B5
:100F10004C05284601F0ACFD58B101A9284601F066
:100F2000DBFCD4F89434024619791868019B00F070
:100F3000B9F803B030BD000000EB8103F7B59C6940
:100F400006460D465CB3202383F3118806EB850724
:100F5000201D0821FFF7A8FEFB685B691B684C3465
:100F600013B1204601F0C6FC204601A901F0B4FCF3
:100F7000024618B130462946019B0BE0FB685A69CE
:100F8000116849B11A8A531E0B4005D130462946D3
:100F900006F1440200F086F8002383F3118803B0C1
:100FA000F0BD0000093138B550F82140DCB12023F4
:100FB00083F31188D4F894241368527903EB8203E5
:100FC000DB689B695D6845B1201D0421FFF76CFE5D
:100FD00004F11400294601F0A1FB2046FFF7B8FEFA
:100FE000002383F3118838BD7047000000F054BF20
:100FF0000123037000234360C36183620362C36201
:1010000043620363038143817047000038B504469F
:10101000202383F3118800254160C5600561456187
:10102000856100F049FF0223237085F3118838BDE4
:1010300070B500EB810306465069DA600D46144630
:1010400018B100211022FFF7F1FDA06918B10021AD
:101050001022FFF7EBFD30462946BDE8704000F056
:10106000F3BF0000028902F001020281428902F00E
:1010700001024281002202614261826101F07AB87C
:10108000F0B500EB81044689E4680125A4698D4030
:101090003543458123600023A2606360BDE8F040D2
:1010A00001F094B8F0B500EB81040689E4680125ED
:1010B00064698D403543058123600023A26063602D
:1010C000BDE8F04001F00EB970B5022300250446DA
:1010D0000370A0F84C5080F84E5080F84F500581B6
:1010E0004581C56005614561856180F8345000F037
:1010F00045FF63681B6823B120462946BDE8704060
:10110000184770BD436802781B6880F8502005229C
:1011100002700BB10421184770470000436890F833
:1011200050201B6802700BB1052118477047000062
:10113000F8B590F83430044613B1002380F8343009
:10114000204604F1440201F037F863689B6833B924
:1011500094F8443013F0600640F0F68005E0204635
:101160009847002840F00281F2E794F8455003F0D8
:101170007F0343EA052540F202339D4200F0D3800D
:1011800014D8022D00F0A48004D855B3012D00F02E
:101190009880D9E0B5F5817F00F0B480B5F5407F47
:1011A00030D0B5F5807F40F0CF8021E040F2016380
:1011B0009D4206D8B5F5C06F4AD2B5F5A06F2FD0C5
:1011C000C2E0B5F5106F58D040F602439D4278D08A
:1011D000B5F5006F40F0B88004F14F03A36301231D
:1011E00049E004F14C03A3630223E3632564BDE0FB
:1011F00094F84630012B40F0A780B4F84C3023F02F
:10120000020308E094F84630012B40F09D80B4F8CA
:101210004C3043F00203A4F84C30A663E6636FE061
:10122000B4F84430B3F5A06F0ED194F8463084F88A
:101230004E30204600F0FCFE63681B6813B1204668
:1012400001219847032323700023A363E3633DE058
:10125000626894F8497094F84830556894F84710DB
:1012600094F84620204643EA0723A84700286BD07D
:101270004368A3630368E36342E02378042B10D13F
:10128000202383F311882046FFF7ECFE86F31188B4
:10129000636884F84F601B68032121700BB12046FE
:1012A000984794F84630002BCED084F84F30042372
:1012B000237063681B68002BC6D020460221984724
:1012C000C2E74E4BA3630223E363002323644DE094
:1012D00094F8481011F0800F204601F00F0102D061
:1012E00000F05CFF01E000F04BFF012805D0022870
:1012F0002AD1434BA363E06302E0424BA363E5635F
:10130000266433E094F84630F3B994F8483013F08B
:101310000F0199D01A06204602D501F0B1F993E7E2
:1013200001F0A4F990E794F846306BB994F848308E
:1013300013F00F0188D01B06204602D501F08CF96E
:1013400082E701F07FF97FE72046002101F084F970
:101350002046002101F076F963681B6813B120462E
:1013600006219847062384F83430F8BD94F84B20C2
:1013700094F84A3043EA0223E26B9A4288BFE3635F
:1013800094F94430E16B002B0D464FF0200317DA3F
:1013900059B1092284F8342083F3118800212046B2
:1013A000A26BE36BFFF77EFE16E0142284F8342074
:1013B00083F3118820460A460B46FFF761FE19E0C9
:1013C00071B1152284F8342083F31188002120465E
:1013D000A26BE36BFFF754FE002383F31188F8BD83
:1013E0000B2284F8342083F3118820460A460B46EA
:1013F000FFF758FE85F31188F8BD00BFC43200081E
:10140000C8320008CC32000838B590F834300446B1
:10141000152B4DD8DFE803F03C4C4C4C4C4C3C4C6D
:101420004C0B27374C4C4C4C4C4C4C4C3C3C90F8A7
:101430004B1090F84A30C26B43EA01239A4212D211
:10144000C3681D8AB2FBF5F305FB13255DB92023A4
:1014500083F3118829462A462B46FFF723FE85F39E
:1014600011880A2322E0142384F83430202383F3E4
:10147000118800210B4620460A46FFF701FE002393
:1014800083F3118838BD036C03B1984700230DE046
:10149000002101F0E1F82046002101F0D3F8636853
:1014A0001B6813B1204606219847062384F8343080
:1014B00038BD000090F83420152A38B5044631D8DC
:1014C0000123934040F641621A40DAB913F48015C3
:1014D0000FD19B0226D50B2380F83430202383F3D1
:1014E000118829462A462B46FFF7DCFD85F3118833
:1014F00038BDC3689B695B68A3B9036C03B19847A7
:1015000000230DE0002101F0A7F82046002101F0A2
:1015100099F863681B6813B1204606219847062393
:1015200084F8343038BD0000024B00221B605B6041
:101530009A607047600D0020002303748268054B99
:101540001B6899689142FBD25A6803604260106040
:1015500058607047600D002008B5202383F3118880
:10156000037C032B03D0042B05D04BB90EE0436959
:1015700000221A6004E090E80C001A6002685360D0
:101580004FF0FF334361FFF7D7FF002383F3118848
:1015900008BD0000002303748268054B1B6899682E
:1015A0009142FBD85A6803604260106058607047EF
:1015B000600D0020054B19690874186802681A60EC
:1015C0005360186101230374FEF79EBE600D002076
:1015D00030B54B1C87B005460A4C0DD023690A4A2A
:1015E00001A800F0D3F82846FFF7E4FF049B2BB1D5
:1015F00001A800F007F901E0FFF7DCFF2369586953
:1016000007B030BD600D00205915000838B50C4DED
:1016100041612B6981689A689142044603D8BDE80C
:101620003840FFF789BF1846FFF786FF01232C617A
:10163000014623742046BDE83840FEF765BE00BF72
:10164000600D0020044B1A681B6990689B689842E3
:1016500094BF002001207047600D002010B5084C99
:10166000236820691A6822605460012223611A7479
:10167000FFF790FF01462069BDE81040FEF744BE29
:10168000600D0020826002220274002242747047C2
:101690008368A3F17C0243F80C2C026943F83C2CCC
:1016A000426943F8382C074A43F81C2CC26843F8B7
:1016B000102C022203F8082C002203F8072CA3F1B7
:1016C000180070472103000810B5202383F3118808
:1016D000FFF7DEFF00210446FFF798FF002383F3A6
:1016E0001188204610BD0000024B1B6958610F2075
:1016F000FFF760BF600D0020202383F31188FFF700
:10170000F3BF000008B50146202383F311880820A9
:10171000FFF75EFF002383F3118808BD49B1064B34
:1017200042681B6918605A60136043600420FFF729
:101730004FBF4FF0FF307047600D002003688342B9
:1017400006D01A680260506059611846FFF7F4BE6F
:101750007047000038B504460D462068A04206D008
:10176000036823605C604561FFF7E6FEF5E738BD7E
:10177000054B03F114025A619A614FF0FF32DA61AE
:1017800000221A62704700BF600D0020F8B50361A7
:101790004FF08043C2605C6A194B1A46012998BF1A
:1017A000022152F8145F954206461F460AD158613D
:1017B00098611C620560456081600819BDE8F840C9
:1017C00001F076B9186AAB68241A0C1905D29C424C
:1017D00005D2204401F07AF901E02D68E41AAB68E3
:1017E000A342FAD36B68736035601E606E60B460AC
:1017F000A9684FF0FF33091BA960FB61F8BD00BF6A
:10180000600D002010B51A4C234653F8141F814276
:101810000ED0416802680A60026851609A424FF037
:101820000001C16023D0916883680B44936010BDB0
:101830000A68626100209A425360C86003D1BDE823
:10184000104001F03DB988689368034493604FF0FD
:101850008042206A526A121A9A4208D2991A0129C1
:1018600098BF931C1844BDE8104001F02FB910BD7B
:10187000600D002000207047FEE700004FF0FF30B1
:1018800070470000022906D0032906D00129064826
:1018900018BF0020704705487047032A9ABF044BC1
:1018A00003EBC20000207047DC330008F43200086C
:1018B0000808002070B5044608460D46FFF7AEF94B
:1018C00006462046013403783BB12946F2B2FFF7C1
:1018D0008DF90028F5D1012070BD184670BD0000BB
:1018E0002DE9F04307469BB008460C461646FFF725
:1018F00095F93D49C5B22046FFF7DCFF08B1063532
:10190000EDB220463949FFF7D5FF08B11035EDB2E9
:10191000632D0DF1040801DC45461BE040462146DD
:1019200001F02CFC41E0B9F1250F37D120462E49BA
:101930000722FFF75BF998B92D4B2A4603F10C01FA
:1019400053F8040B42F8040B8B42F9D11B78137047
:1019500007340D3594F80090B9F1000FE3D122E07F
:10196000204622490822FFF741F9B8B92149AB1CAA
:1019700011F8012F20484FEA121E02F00F021EF844
:1019800000E0125C03F8012C1C4A03F802EC9142BF
:1019900003F10203ECD118350834DBE785F8009039
:1019A00001340135D6E785F800904046FFF736F957
:1019B000C0B2431C5B0087E8480033700323737098
:1019C00002360023DAB2824206F1020608D218F883
:1019D000032006F8022C002206F8012C0133F1E75F
:1019E0001BB0BDE8F08300BF203300082833000897
:1019F000313300080F7AFF1F3F3300081B7AFF1FA7
:101A000008B5202383F311880348FFF76FFA0023FA
:101A100083F3118808BD00BFB00D002010B5044647
:101A2000052924D8DFE801F013230313131A202318
:101A300083F3118801210E4AFFF7FAFA20460221AA
:101A40000C4AFFF7F5FA0C48FFF716FA0CE02023D2
:101A500083F311880848FFF7EBF905E0202383F3AF
:101A600011880548FFF7FCF9002383F3118810BDA6
:101A7000D0320008FC320008B00D002038B50C4D03
:101A80000C4C0D4905F108002246FFF729FF05F12E
:101A9000100004F1CA020949FFF722FF05F11800FE
:101AA00004F5CA720649BDE83840FFF719BF00BF08
:101AB0000808002068120020503300085A3300083C
:101AC00028330008BFF34F8F024BDB68DB03FBD4E6
:101AD000704700BF003C024008B5094B1B7873B942
:101AE000FFF7F0FF074B1A69002ABFBF064A5A608A
:101AF00002F188325A601A6822F480621A6008BDC6
:101B0000F9140020003C02402301674508B50B4B47
:101B10001B7893B9FFF7D6FF094B1A6942F00042D0
:101B20001A611A6842F480521A601A6822F48052CC
:101B30001A601A6842F480621A6008BDF914002025
:101B4000003C02400B2830B513D80B4A0B4C1378DD
:101B500063B94FF000610A4D44F8231055F8235043
:101B600001330C2B2944F6D10123137054F82000C3
:101B700030BD002030BD00BFF8140020C814002084
:101B8000E4330008014B53F820007047E4330008A9
:101B90000C2070470B2810B5044601D9002010BD59
:101BA000FFF7D0FF064B53F824100A4643189B1A40
:101BB00022B11B680133F1D1043AF7E7012010BDCF
:101BC000E43300080B2838B5044621D8114DFFF73F
:101BD00079FFFFF781FFF323EB60FFF773FF0C2220
:101BE000B4FBF2F302FB1343DB00DBB243F40073FC
:101BF00043F002032B612B6943F480332B61FFF721
:101C000061FFFFF783FF2046BDE83840FFF7C2BF02
:101C1000002038BD003C02402DE9F84F1446E20791
:101C2000074689466ED42318B3F1016F6AD2374B49
:101C30001B68DB0766D5FFF74FFF354BF322DA60F1
:101C4000FFF740FF4E46A246C9EB0708BAF1030F63
:101C5000B346B04401D8B14624E018F0030FFAD1DE
:101C60002B4D2B6923F440732B612B6943F40073D4
:101C700043F001032B613368C8F80030BFF34F8F86
:101C8000FFF720FFEB6813B1F323EB602BE0D8F8EC
:101C90000080DBF80030984506F1040623D1AAF154
:101CA000040AD1E7C9EB0A033344194DC6EB080710
:101CB000012B4F442B691DD923F440732B612B69F1
:101CC00043F4807343F001032B61CB4639F8023BA8
:101CD0003B80BFF34F8FFFF7F5FE3F88BBF8003026
:101CE000BFB2BB42DED02B6923F001032B61FFF7AB
:101CF0000DFF07E023F001032B61FFF707FF2046EC
:101D0000BDE8F88F4FF0FF30BDE8F88F0038024093
:101D1000003C024010B5084C237828B153B9FFF7B6
:101D2000DBFE0123237010BD23B12070BDE81040FD
:101D3000FFF7ECBE10BD00BFF9140020014B186D79
:101D4000704700BF002800400A4B1A6F12045FBFA3
:101D50001A6F42F400721A671A6F5CBF42F40042B5
:101D60001A67054A136843F480731360034B1865C0
:101D7000704700BF0038024000700040002800405B
:101D800070470000FEE70000084A094B09498B42F2
:101D900004D252F8041F43F8041BF7E7064A9342A3
:101DA00003D2002243F8042BF8E770478C35000873
:101DB000F0170020F0170020F0170020836D30B5D9
:101DC000446D9D68002204EB4213013200214FF064
:101DD000FF30AA42C3F80019C3F81019C3F8080964
:101DE000C3F8001BC3F8101BC3F8080BEBD94FF066
:101DF0000113C4F81C3830BD890141F02001016194
:101E000003699B06FCD4122000F0EABE2DE9F043E2
:101E1000204D05EB8003D5F85490D3F80CC0DCF8C6
:101E2000142000F1010ED2F8008009EB0E3E51683B
:101E300041450CD3696D0123D1F8342803FA00F031
:101E400022EA0002C1F834281846BDE8F083BCF845
:101E50001040C1EB0803A34228BF234609EB4014FE
:101E6000D4F81849A4B2B3EB840F0FD8946826466F
:101E70003768CEF800709F1B2744042F01D9043621
:101E8000F6E71C440B4494605360D0E70020BDE8A3
:101E9000F08300BFFC14002010B5054C2046FFF76E
:101EA000A7F84FF0A0436365024BA36510BD00BFC8
:101EB000FC140020143400080378012B70B505468B
:101EC000446D4ED1274B98421BD1274B5A6B42F0A1
:101ED00080025A635A6D42F080025A655A6D5A69FF
:101EE00042F080025A615A6922F080025A6143200E
:101EF0000E215B6900F0CEFB1C4BE3601C4BC4F869
:101F000000380023C4F8003EC02323604FF40413BC
:101F1000A3636E6D202000F063FE012333613369FB
:101F2000DB07FCD4122000F05BFE3369002BFCDAE7
:101F30000026A6602846FFF741FF6B68C4F81068CA
:101F4000DB68C4F81468C4F81C680BB9094B00E0DE
:101F5000094BA3614FF0FF336361A36843F00103B2
:101F6000A36070BDFC140020003802404014004003
:101F700003002002003C30C0083C30C070B5446D06
:101F8000054600212046FFF737FFA96D00234FF0DB
:101F900001128E68C4F83438C4F81C2804EB4312CC
:101FA0004FF000600133C2F80009B342C2F8000BE1
:101FB0004FF0FF30C2F80809C2F8080BEED90B68E1
:101FC000EB656A6D0B68636210231361136913F08C
:101FD0001006FBD1122000F003FED4F8003823F4E1
:101FE000FE63C4F80038A36943F4402343F01003B0
:101FF000A3610923C4F81038C4F814380A4BEB6005
:102000004FF0C043C4F8103B084BC4F8003BC4F881
:102010001069C4F80039EB6D03F1100243F480132A
:10202000EA65A36270BD00BF203400084080001044
:10203000426D90F84E10D2F8003823F4FE6343EA64
:102040000113C2F8003870472DE9F0410FB200EBE0
:1020500087080D46D8F80C10446D0E6806F003038F
:10206000022B07D0032B07D03D4A3E4E012B18BF51
:10207000164602E03C4E00E03C4E6A01A3184FF0C9
:10208000000EC3F810EB8B6905F1100C8BB1B1F8A1
:1020900012E005F158035B0146EA0E0E44F803E036
:1020A0004FF0010ED4F81C380EFA0CFE4EEA030372
:1020B0000FE004EB471EDEF8003B23F40043CEF8AC
:1020C000003BD4F81C384FF0010E0EFA0CFE23EA48
:1020D0000E032244C4F81C380023C2F810394B699F
:1020E00005F13F020BB30B8A898B9B08012988BF3E
:1020F0004B43C16D04EB82025F1841EA0343C7659D
:10210000294653602046FFF777FED8F80C301B8A2B
:1021100043EA85531E4305F148035B01E650012362
:10212000D4F81C28AB40134315E004EB8202104B9B
:10213000536020462946FFF75FFE04EB4713D3F8B0
:10214000002922F40042C3F80029D4F81C280123F6
:10215000AB4022EA0303C4F81C38BDE8F08100BF9D
:1021600000800010008004100080081000800C1017
:1021700000040002826D1268C265FFF71FBE0000F6
:102180005831436D49015B5813F4004004D013F4F7
:10219000001F14BF01200220704700004831436D2A
:1021A00049015B5813F4004004D013F4001F14BF1E
:1021B000012002207047000000EB8101CB68196A02
:1021C0000B6813604B6853607047000000EB81039D
:1021D00030B5DD68AA691368D36019B9402B84BF94
:1021E0004023136014686B8A426D013C1C44B4FBAD
:1021F000F3F46343E004033340F0C04023F00303EF
:10220000034302EB411009B2C0F8103B2B6803F006
:102210000303012B0ED1D2F8083802EB411013F45E
:10222000807FD0F8003B14BF43F0805343F000534D
:10223000C0F8003B02EB4112D2F8003B43F00443EC
:10224000C2F8003B30BD00002DE9F041244D6E6D19
:1022500006EB40130446D3F8087BC3F8087B380725
:102260000AD5D6F81438190706D505EB8403284695
:10227000DB6821465B689847FA072ED5D6F81438F4
:10228000DB072AD505EB8403D9688B69C4B94A8A70
:102290005E68B6FBF2F002FB10628AB91868DA6871
:1022A00090420DD2121A83E81400202383F3118880
:1022B0000B482146FFF78AFF84F31188BDE8F081BF
:1022C0006A890123A34022EA03036B81CB6823B10F
:1022D00021460348BDE8F0411847BDE8F08100BF42
:1022E000FC14002000EB8103F0B5DD68436D6A69E2
:1022F0001668D6604C011EB91C444FF400220FE052
:1023000019B9402E84BF4020106012682F8A42F015
:102310000056013AD0191C44B0FBF7F246EAC2421B
:10232000C4F810292A6802F00302012A0AB20ED169
:10233000D3F8080803EB421410F4807FD4F80009A6
:1023400014BF40F0805040F00050C4F8000903EB87
:102350004212D2F8000940F00440C2F80009D3F854
:10236000340801228A400243C3F83428F0BD00003B
:10237000F8B504461D48456D05EB4413D3F80869CC
:10238000C3F80869F10722D5D5F81038DA071ED549
:1023900000EB8403D9684B691F68DA6897420CD256
:1023A000D21B00271A605F60202383F31188214627
:1023B000FFF798FF87F3118809E002890123A34002
:1023C00022EA030303818B680BB121469847330649
:1023D0000AD5D5F834280123A340134204D020465F
:1023E000BDE8F840FFF712BDF8BD00BFFC140020A7
:1023F00093482DE9F843446D6369A5691D4015F4C0
:10240000805F6561064602D0FEF75EFE13E1002D97
:1024100012DAD4F8003E8A489B071EBFD4F8003E6B
:1024200023F00303C4F8003ED4F8043823F001037A
:10243000C4F80438FEF772FE2F0502D58048FEF777
:1024400061FEA8040CD5D4F8083813F0060FE36831
:1024500023F470530CBF43F4105343F4A053E360D0
:10246000290704D57368DB680BB175489847EA0201
:1024700002D4AB0243D538E0D6F854904FF00008B0
:10248000B36D9B685FFA88F79F42F2D809EB471358
:10249000D3F8002902F44022B2F5802F22D1D3F8DC
:1024A0000029002A1EDAD3F8002942F09042C3F82E
:1024B0000029D3F80029002AFBDB706D3946FFF7AD
:1024C0009BFC32890123BB4022EA0303338106EBE4
:1024D0008703DB689B6813B15948394698473846EB
:1024E000FFF794FC08F10108CAE7776D4FF0000888
:1024F000B36D53489B685FFA88F1994202D9EF06A1
:102500006BD51BE007EB4112D2F8003B03F44023EC
:10251000B3F5802F0FD1D2F8003B002B0BDA4289A4
:1025200001238B4022EA0303438100EB8103DB6834
:10253000DB6803B1984708F10108D9E7706D404B9B
:10254000026AC2F30A1702F00F0102F4F012B2F5A8
:10255000802F18D0B2F5402F3FD103EB8103DB6809
:10256000196A00231A46BB4237D09E0704BF00F504
:1025700080521268072B98BF0A7003F101039CBFB9
:10258000120A0131EFE78A1C03EB82035B68996949
:102590000B68D1F808C04968C1EB030E0023194647
:1025A000BB4210D013F0030F04BF00F5805109683F
:1025B000734538BF8CF8001003F101033CBF090AD2
:1025C0000CF1010CECE706EB8206726892699168E7
:1025D0001944916051680B4453602903D4F818489A
:1025E00013D5E20302D50020FFF72EFEA30302D588
:1025F0000120FFF729FE670302D50220FFF724FE22
:10260000260302D50320FFF71FFE6D0313D5E00755
:1026100002D50020FFF7ACFEA10702D50120FFF78D
:10262000A7FE620702D50220FFF7A2FE230702D50C
:102630000320FFF79DFEBDE8F84300F063BB00BF39
:10264000FC140020436D03EB4111D1F8003B43F42F
:102650000013C1F8003B7047436D03EB4111D1F803
:10266000003943F40013C1F800397047436D03EBA0
:102670004111D1F8003B23F40013C1F8003B70472F
:10268000436D03EB4111D1F8003923F40013C1F875
:102690000039704700F1604300F01F02400903F564
:1026A000614309018000C9B200F1604083F8001362
:1026B00000F5614001239340C0F88031036070470A
:1026C00030B5039C0172043304FB0325C361049BF2
:1026D00003630021059B00604060C16042610261AC
:1026E0008561046242628162C162436330BD000061
:1026F0000022416A41610161C2608262C2626FF080
:102700000101FFF727B8000003694269934203D132
:10271000C2680AB100207047181D704710B50469DF
:102720002160C268C3690132C26082692344934256
:10273000036124BF436A03610021BDE81040FEF736
:10274000FDBF000038B504460D46E36843B9237A5F
:1027500073B920462946FEF7E1FF0028F5DA09E0C3
:1027600063691A1D1B68A2621344E362002038BD2E
:102770006FF0010038BD0000C3684269013BC360CF
:10278000C369134482694361934224BF436A43612E
:1027900000238362036B03B11847704738B50546C1
:1027A000202383F31188846A2CB9FFF7CBFF10B183
:1027B00084F3118838BDAB6AEA6A13F8014BAB6247
:1027C000934202D32846FFF7D7FF002383F31188F3
:1027D000204638BD2DE9F0471F4604460E46914677
:1027E000202383F311884FF080434FF0000A5B6A87
:1027F00007EB0308A36AA3B97A1E033202D9204665
:10280000394607E04FF08042516AC1EB0801B942F6
:1028100004D82046FFF796FF18B1002383F31188F0
:1028200032E0A16AE56ACAEB09036D1A9D4228BF2E
:102830001D46402D0FD9334601F1400251F8040BDB
:1028400043F8040B9142F9D1A36A40334036A362A6
:102850000AF1400A08E030462A46FEF7BDF9A36AAD
:102860002B442E44A362AA44A26AE36A9A4202D38A
:102870002046FFF781FF002383F31188CA4503D266
:10288000202383F31188B5E75046BDE8F0870000A8
:1028900010B5029C0172043303FB0421C3610023C1
:1028A0008362C362039B0363049B00604060C46057
:1028B00042610261816104624262436310BD0000B3
:1028C000026AC260426A4261026100228262C2629E
:1028D0006FF00101FEF73EBF436902699A4203D1DE
:1028E000C2680AB100207047184650F8043B0B60DC
:1028F00070470000C36842690133C360C369134471
:1029000082694361934224BF436A43610021FEF719
:1029100015BF000038B504460D46E36843B9237A75
:1029200073B920462946FEF7F9FE0028F5DA09E0DA
:102930002269131DA362E3691344E362002038BDDA
:102940006FF0010038BD000010B504692160C26855
:10295000C369013AC260826923449342036124BF80
:10296000436A036100238362036B13B1BDE8104027
:10297000184710BD70B5202304460E4683F3118816
:10298000856A35B91146FFF7C5FF10B185F3118887
:1029900070BDA36A1E70A36AE26A01339342A36208
:1029A00004D3E16920460439FFF7CEFF002080F30D
:1029B000118870BD2DE9F0471F4604460D4691462B
:1029C000202383F311884FF080434FF0000A5B6AA5
:1029D00007EB0308A36AA3B97A1E033202D9204683
:1029E000394607E04FF08042516AC1EB0801B94215
:1029F00004D82046FFF78EFF18B1002383F3118817
:102A000032E0A06AE66ACAEB0903361A9E4228BF82
:102A10001E46402E0DD905F1400355F8042B40F811
:102A2000042B9D42F9D1A36A4033A3620AF1400A04
:102A300008E029463246FEF7CFF8A36A334435440E
:102A4000A362B244A26AE36A9A4204D3E1692046CF
:102A50000439FFF779FF002383F31188CA4503D2B5
:102A6000202383F31188B5E75046BDE8F0870000C6
:102A7000026943699A4203D1C3680BB1836A0BB9F7
:102A800000207047043B9B1AFAD01360C368013BD7
:102A9000C360C3691A44836902619A4224BF436ACE
:102AA00003610023836201207047000000F06CB9CD
:102AB0004FF08043002258631A610222DA607047A7
:102AC0004FF080430022DA60704700004FF08043EF
:102AD00058637047FEE7000010B5174CFEF724FD61
:102AE000FEF746FE204615498022FEF7CBFD012366
:102AF00044F8180C0374124B124AD96821F4E061AF
:102B00000904090C0A431049DA60CA6842F080726D
:102B1000CA600E490A6842F001020A601022DA77A0
:102B2000202283F82220002383F3118862B608480C
:102B3000BDE81040FEF7C8BD880D002044340008F1
:102B400000ED00E00003FA05F0ED00E0001000E009
:102B5000503400082DE9F843204D6C69A2681F49E4
:102B60004FF0804301F11408586A2B6AC61A964246
:102B70001ED3A2682B6AD4F80C901344B61A2268AC
:102B80002B6242454FF00003C2F804801F466A6181
:102B9000E36001D1FFF794FF87F311882069C847EC
:102BA000202383F311886C69A368B342E1D9D5E788
:102BB0004A6942450FD033440B6291688E1B966080
:102BC000A2681B1A1344012B98BF02231844BDE8C6
:102BD000F843FFF77BBFBDE8F88300BF600D00201E
:102BE000034B59685A68521A8242FBD3704700BFA0
:102BF000001000E04B6843608B688360CB68C36063
:102C00000B6943614B6903628B6943620B68036024
:102C100070470000224B2348196940F2FF1211430C
:102C200010B519611969204C21F4FF7121F00101DF
:102C300019611969196B11431963196D0A431A65F2
:102C400021461B6DFFF7D6FF04F11C011748FFF763
:102C5000D1FF04F138011648FFF7CCFF04F154010D
:102C60001448FFF7C7FF04F170011348FFF7C2FFD4
:102C700004F18C011148FFF7BDFF04F1A8011048D1
:102C8000FFF7B8FF04F1C4010E48FFF7B3FF04F1EA
:102C9000E0010D48FFF7AEFFBDE8104000F0DEB8E0
:102CA000003802400000024068340008000402407E
:102CB00000080240000C02400010024000140240D4
:102CC00000180240001C02400020024008B500F03D
:102CD00039FAFFF701FFBDE80840FEF7CFBE00005C
:102CE00070470000064A536823F001035360EFF376
:102CF0000983683383F30988002383F311887047BD
:102D000030EF00E010B5202383F31188104B5B688F
:102D100013F4006318D0F1EE103AEFF309844FF08A
:102D2000807344F84C3C0B4BDB6844F8083CA4F13E
:102D3000680383F30988FEF785FC08B1064B00E0C1
:102D4000064B44F8503C10BD83F3118810BD00BF02
:102D500000ED00E030EF00E031030008340300082C
:102D60004FF0804310B51A69920708D500241C6102
:102D7000202383F31188FFF7EDFE84F31188BDE86B
:102D80001040FFF7BFBF0000104B1A6C42F0010269
:102D90001A641A6E42F001021A660D4A1B6E93689D
:102DA00043F0010393604FF0804353229A624FF047
:102DB000FF32DA6200229A615A63DA605A600122B5
:102DC0005A611C201A600821FFF764BC00380240D9
:102DD000002004E01F4B1A696FEAC2526FEAD25218
:102DE0001A611A69C2F308021A614FF0FF301A69BA
:102DF0005A69586100215A6959615A691A6A62F020
:102E000080521A621A6A02F080521A621A6A5A6A68
:102E100058625A6A59625A6A1A6C42F080521A64AD
:102E20001A6E42F080521A661A6E0B4A106840F40D
:102E300080701060186F00F44070B0F5007F1EBF06
:102E40004FF4803018671967536823F40073536098
:102E500000F058B90038024000700040324B4FF08B
:102E600080521A64314A4FF4404111601A6842F0AE
:102E700001021A6019682C4A8807FBD5936823F071
:102E800003039360284B9A6812F00C02FAD1196878
:102E900001F0F90119609A601A6842F480321A60F0
:102EA0001968214A8903FBD5536F43F00103536727
:102EB0001D4B5A6F9007FBD51D4A5A601A6842F0A5
:102EC00080721A60194B5B685904FBD5164B1A685F
:102ED0009201FBD5174A9A60174B1A68174B9A4212
:102EE000174B07D1174A1168174A914202D140F295
:102EF000051201E040F205721A600B4B9A6842F02D
:102F000002029A601A469168074B01F00C010829E9
:102F1000F9D15A6C42F480425A645A6E42F48042AB
:102F20005A665B6E704700BF003802400070004078
:102F30000854400700948838002004E01164002001
:102F4000003C024000ED00E041C20F41084A08B5D4
:102F5000516913680B4003F00103536123B1054A23
:102F600013680BB150689847BDE80840FFF7CABE28
:102F7000003C014070170020084A08B551691368E9
:102F80000B4003F00203536123B1054A93680BB170
:102F9000D0689847BDE80840FFF7B4BE003C014048
:102FA00070170020084A08B5516913680B4003F0F8
:102FB0000403536123B1054A13690BB15069984763
:102FC000BDE80840FFF79EBE003C0140701700209E
:102FD000084A08B5516913680B4003F008035361B0
:102FE00023B1054A93690BB1D0699847BDE8084001
:102FF000FFF788BE003C014070170020084A08B562
:10300000516913680B4003F01003536123B1054A63
:10301000136A0BB1506A9847BDE80840FFF772BECB
:10302000003C014070170020174B10B55A691C680E
:10303000144004F478725A61A30604D5134A936AC3
:103040000BB1D06A9847600604D5104A136B0BB1D8
:10305000506B9847210604D50C4A936B0BB1D06B8B
:103060009847E20504D5094A136C0BB1506C984798
:10307000A30504D5054A936C0BB1D06C9847BDE805
:103080001040FFF73FBE00BF003C0140701700201A
:103090001A4B10B55A691C68144004F47C425A61FA
:1030A000620504D5164A136D0BB1506D9847230580
:1030B00004D5134A936D0BB1D06D9847E00404D545
:1030C0000F4A136E0BB1506E9847A10404D50C4AF9
:1030D000936E0BB1D06E9847620404D5084A136F03
:1030E0000BB1506F9847230404D5054A936F0BB179
:1030F000D06F9847BDE81040FFF704BE003C014088
:1031000070170020062008B50146FFF7C3FA072014
:103110000621FFF7BFFA08200621FFF7BBFA0920B6
:103120000621FFF7B7FA0A200621FFF7B3FA1720A6
:103130000621FFF7AFFA28200621BDE80840FFF777
:10314000A9BA000008B5FFF745FE00F00BF8FDF73F
:103150004DFFFDF725FEFFF7C3FDBDE80840FFF773
:10316000A5BC00000023044A002199501A440833EA
:10317000802B5160F7D170477017002080EA010260
:10318000844612F0030F4FD111F0030F32D14DF8E6
:10319000044D11F0040F51F8043B0BD0A3F10132A0
:1031A0009A4312F0803F04BF4CF8043B51F8043BB3
:1031B00016D100BF51F8044BA3F101329A4312F02B
:1031C000803FA4F101320BD14CF8043BA24312F032
:1031D000803F04BF51F8043B4CF8044BEAD023462F
:1031E0000CF8013B13F0FF0F4FEA3323F8D15DF8E1
:1031F000044B704711F0010F06D011F8012B0CF8A9
:10320000012B002A08BF704711F0020FBFD031F820
:10321000022B12F0FF0F16BF2CF8022B8CF80020A7
:1032200012F47F4FB3D1704711F8012B0CF8012B2A
:10323000002AF9D1704700BF1210121312110000BA
:1032400000000000703200083F000000130400007E
:103250007A3200083F0000001904000084320008A0
:103260003F000000210400008E3200083F000000F3
:1032700053544D3332463F3F3F0053544D33324653
:103280003430780053544D3332463432780053543E
:103290004D333246343436585800000000000000E8
:1032A0001D0D0008090D0008450D0008310D00082E
:1032B0003D0D0008290D0008150D0008010D00083E
:1032C000B90C000800000000000000000100000030
:1032D0000200000000000000390F0008A50F0008E0
:1032E0004000400048120020581200200200000058
:1032F00000000000430000007833000803000000D5
:1033000000000000E90F00080000000010000000AD
:10331000A00D0020000000000100000000000000DF
:1033200025424F41524425002553455249414C25E1
:10333000004F6D6E696275734E616E6F5636003068
:10334000313233343536373839414243444546000B
:103350004172647550696C6F740025424F4152444C
:10336000252D424C000000001D1A00088518000899
:10337000A50E0008011A000809024300020100C05E
:1033800032090400000102020100052400100105B9
:10339000240100010424020205240600010705821D
:1033A000030800FF09040100020A000000070501EC
:1033B00002400000070581024000000012011001D8
:1033C0000200004083044057000201020301000094
:1033D00004030904FC140020010102001200000093
:1033E000BC33000800400000004000000040000026
:1033F0000040000000000100000002000000020088
:1034000000000200000002000000020000000200B4
:1034100000000200800000004001000003000000E6
:10342000000000003111000809140008B51400085C
:10343000400040005C1500205C15002001000000E9
:103440006C1500206D61696E0069646C6500000098
:103450004934000878150020701700200100000092
:10346000D52A0008000000000000810200000000D2
:10347000AAAAAAAA00000000FFFE000000000000A7
:1034800000A00A000000000000000000AAAAAAAAEA
:1034900000000000FFFF000000000000000000002E
:1034A0000000000000000000AAAAAAAA0000000074
:1034B000FFFF00000000000000000000000000000E
:1034C00000000000AAAAAAAA00000000FFFF000056
:1034D00000000000000000000000000000000000EC
:1034E000AAAAAAAA00000000FFFF00000000000036
:1034F000000000000000000000000000AAAAAAAA24
:1035000000000000FFFF00000000000000000000BD
:103510000000000000000000AAAAAAAA0000000003
:10352000FFFF00000000000000000000000000009D
:10353000000000000A00000000000000030000007E
:10354000000000000000000000000000000000007B
:10355000000000000000000000000000000000006B
:103560000000000000000000FF00960000000008BE
:1035700004000000D033000800000000000000003C
:10358000000000000000000000000000000000003B
:00000001FF
